:0200000480007A
:100000006F00C004732F2034930F8000630AFF0336
:10001000930F90006306FF03930FB0006302FF038A
:10002000170F0080130F0FFE63040F0067000F000F
:10003000732F203463540F006F004000136E9E53E3
:10004000171F00002320CFFD6FF09FFF732540F1A5
:100050006310050073251030635805000F00F00F82
:10006000130E100073000000130E00009702000032
:10007000938282F973905230735020307350303035
:1000800073504030970200809382C2F7638C020065
:10009000739052109302B01A739022307323203061
:1000A000E39E62F873500030970200009382420191
:1000B00073901234732540F1730020301300000058
:1000C000172500001305C571EF0540003305B54045
:1000D000B72E0000938E0E71130E20006314D5030B
:1000E00017E5FFFF1305C58FEF0540003305B54049
:1000F000B7EEFFFF938E0E8F130E30006314D50101
:10010000631CC0010F00F00F63000E00131E1E00E1
:10011000136E1E00730000000F00F00F130E10008E
:1001200073000000731000C0000000000000000019
:1001300000000000000000000000000000000000BF
:1010000000000000000000000000000000000000E0
:1010100000000000000000000000000000000000D0
:1010200000000000000000000000000000000000C0
:1010300000000000000000000000000000000000B0
:081040000000000000000000A8
:040000058000200057
:00000001FF
